:100000000C9438000C9455000C9455000C94550039
:100010000C9455000C9455000C9455000C9455000C
:100020000C9455000C9455000C9455000C945500FC
:100030000C9455000C9455000C9455000C945500EC
:100040000C9444010C9455000C9455000C945500EC
:100050000C9455000C9455000C9455000C945500CC
:100060000C9455000C9455000C9455000C945500BC
:1000700011241FBECFEFD0E1DEBFCDBF11E0A0E065
:10008000B1E0EAECFAE002C005900D92A43CB107A1
:10009000D9F712E0A4ECB1E001C01D92A432B1077F
:1000A000E1F70E9403020C9463050C94000087E6BC
:1000B0008093C40088E18093C10008951F93182F96
:1000C000873049F4609122027091230280E091E030
:1000D0000E9484020BC08A3019F48DE00E945E00F9
:1000E0008091C00085FFFCCF1093C60080E090E0B7
:1000F0001F910895EF92FF920F931F93CF93DF9379
:100100007C018091C4019091C501892B09F0A0C0A8
:1001100006EC11E08091C00087FFFCCF8091C00009
:1001200084FF03C02EEF3FEFA7C08091C00083FD86
:10013000A1C09091C6009D3011F09A3069F48AE018
:10014000F8018083B7010E945E0086EC91E09093F5
:10015000C5018093C4017CC0993009F490E2892FD5
:1001600080528F3510F0903A78F0F2E005311F0799
:1001700019F4B70187E005C0F80191938F01B70129
:10018000892F0E945E00C6CF923139F1933138F445
:10019000933009F46FC0983009F0BCCF09C0973193
:1001A00009F44BC09F3721F0953109F0B3CF32C02D
:1001B000F1E0063C1F0709F008F4ACCFB70188E076
:1001C0000E945E00B70180E20E945E00B70188E0F5
:1001D0000E945E00015010409DCFB7018DE00E944B
:1001E0005E00C6ECD1E004C0B70189910E945E00B8
:1001F000C017D107C8F38ECFB70188E00E945E0018
:10020000B70180E20E945E00B70188E00E945E00B4
:100210000150104081E0063C180709F068F77ACFDA
:10022000B70188E00E945E00B70180E20E945E0094
:10023000B70188E00E945E008E01E1E0063C1E07E7
:1002400009F008F467CFE8018A91803249F762CF5C
:10025000E091C401F091C5018191F093C501E09353
:10026000C4018A3021F41092C5011092C401282FD4
:1002700030E002C02FEF3FEFC901DF91CF911F9116
:100280000F91FF90EF9008951F920F920FB60F926B
:1002900011248F9380911802882329F080911802ED
:1002A00081508093180280911D02882329F080914B
:1002B0001D02815080931D0280911C02882329F029
:1002C00080911C02815080931C028F910F900FBE71
:1002D0000F901F90189580911B02882331F0809118
:1002E000180286958695809318028091170291E0F6
:1002F00089278093170285B908958FE084B915B8CE
:1003000082E08AB980936E009AEF97BD84BD83E046
:1003100085BD8FEF80931702909318028DE780932D
:100320001D028CE380931C0284E0809316021092DD
:100330001B020E94570066E471E0709323026093F1
:10034000220270931F0260931E0270932102609339
:10035000200288E091E00E9484027894089589B197
:100360008095807880931B024E990AC026E131E087
:1003700047E650E066E271E084E591E00E943602D3
:100380000895809116028150809316028823D1F53A
:1003900084E0809316028091170292E0892780936F
:1003A000170285B98091190290911A0201969093D3
:1003B0001A028093190201979F938F9388E391E02B
:1003C0009F938F9380912002909121029F938F930E
:1003D0000E9471028DB79EB706960FB6F8949EBF25
:1003E0000FBE8DBF8091190290911A020A9750F0AA
:1003F0002EE331E04AE550E066E271E08AE591E003
:100400000E9436020895EF92FF920F931F930E946D
:100410007D018AEFE82EFF24F3940DE71CE3809121
:100420001802882391F4E092180280911B0288231D
:1004300031F08091180286958695809318028091FC
:1004400017028F258093170285B980911D0288239A
:1004500021F400931D020E94C10180911C02882397
:10046000F1F610931C020E94AF01D9CF0097B1F4AE
:100470005F934F937F936F933F932F9380E691E029
:100480009F938F9380912202909123029F938F9349
:100490000E9471028DB79EB70A9617C05F934F9363
:1004A0007F936F939F938F933F932F938BE891E06C
:1004B0009F938F9380912202909123029F938F9319
:1004C0000E9471028DB79EB70C960FB6F8949EBF2E
:1004D0000FBE8DBF0E946C0281E090E0F8940C94F6
:1004E0006305A0E0B0E0E7E7F2E00C943C05CE0144
:1004F0000996AC016F8178858D819E810E94AD0245
:100500002096E2E00C945805EF92FF920F931F9310
:10051000CF93DF937C018B01DB0113968C9181FDDE
:1005200003C0CFEFDFEF13C0C0E0D0E00BC0D801B5
:100530001896ED91FC911997B8010995892B11F046
:10054000CFEFDFEFF70181917F01882381F7CE01A3
:10055000CDB7DEB7E6E00C945405ABE0B0E0E3EBDA
:10056000F2E00C942C053C012B015A01FC0117828E
:100570001682838181FD03C06FEF7FEFC8C19AE0CF
:10058000892E1E010894211C311CF3012381F201E4
:1005900023FD859123FF81912F01882309F4B4C1A4
:1005A000853239F423FD859123FF81912F01853216
:1005B00029F4B30190E00E94A204E7CF982FDD2434
:1005C000CC249924FFE1FD15D0F09B3269F09C32D8
:1005D00028F4903259F0933291F40EC09D3249F0D4
:1005E000903369F441E024C052E0D52A84E0D82A4F
:1005F00028C098E0D92A25C0E0E1DE2A22C0D7FC35
:1006000029C0892F80538A3070F4D6FE05C0989C8B
:10061000902C1124980E15C0C89CC02C1124C80E13
:10062000F0E2DF2A0EC09E3229F4D6FC6DC140E410
:10063000D42A07C09C3619F450E8D52A02C098364F
:1006400049F4F20123FD959123FF91912F01992304
:1006500009F0B8CF892F8554833018F08052833049
:1006600038F444E050E0A40EB51E5FE359830FC098
:10067000933631F0933779F0933509F056C020C0A6
:10068000F5018081898342E050E0A40EB51E71011E
:1006900001E010E012C0F501E080F180D6FC03C05B
:1006A0006FEF7FEF02C0692D70E042E050E0A40ED2
:1006B000B51EC7010E9497048C015FE7D52214C0C4
:1006C000F501E080F180D6FC03C06FEF7FEF02C040
:1006D000692D70E042E050E0A40EB51EC7010E94F3
:1006E0008C048C0150E8D52AD3FE07C01AC0B30190
:1006F00080E290E00E94A204CA948C2D90E008173A
:100700001907A8F30EC0F701D7FC8591D7FE819198
:100710007F01B30190E00E94A204C110CA9401506D
:1007200010400115110579F7ECC0943611F0993697
:1007300071F5D7FE08C0F501E080F18002811381D8
:1007400044E050E00AC0F501808191817C010027DE
:10075000F7FC0095102F42E050E0A40EB51E5FE6B6
:10076000D52217FF0AC010950095F094E094E11C83
:10077000F11C011D111D80E8D82A2AE030E0A101FA
:10078000C801B7010E94CE04F82EF21840C0953778
:1007900029F41D2D1F7E2AE030E01DC01D2D197F7C
:1007A0009F3661F0903720F4983509F0ADC00FC046
:1007B000903739F0983709F0A7C004C028E030E03E
:1007C0000AC0106114FD146020E130E004C014FD83
:1007D000166020E132E017FF08C0F50160817181E9
:1007E0008281938144E050E008C0F50180819181CD
:1007F000BC0180E090E042E050E0A40EB51EA101F3
:100800000E94CE04F82EF2188FE7D82ED122D6FE01
:100810000BC05EEFD522F91438F4D4FE07C0D2FC29
:1008200005C08FEED82202C01F2D01C0192DD4FEA5
:100830000DC0FE01EF0DF11D8081803319F499EE9A
:10084000D92208C01F5FD2FE05C003C08D2D867857
:1008500009F01F5F0D2DD3FC14C0D0FE0FC01C1576
:1008600010F09F2C0BC09F2C9C0C911A1C2D06C0C5
:10087000B30180E290E00E94A2041F5F1C15C0F348
:1008800004C01C1510F4C11A01C0CC2404FF10C010
:10089000B30180E390E00E94A20402FF1EC001FDAC
:1008A00003C088E790E002C088E590E0B3010CC087
:1008B000802F867891F001FF02C08BE201C080E2B8
:1008C000D7FC8DE2B30190E00E94A20406C0B30100
:1008D00080E390E00E94A2049A94F914C0F3FA9481
:1008E000F101EF0DF11DB301808190E00E94A2049F
:1008F000FF20A9F706C0B30180E290E00E94A204A5
:10090000CA94CC20C1F741CEF30166817781CB0137
:100910002B96E2E10C944805FC0105906150704073
:100920000110D8F7809590958E0F9F1F0895FC01B8
:100930006150704001900110D8F7809590958E0F0E
:100940009F1F08950F931F93CF93DF938C01EB01AB
:100950008B8181FF1BC082FF0DC02E813F818C8166
:100960009D812817390764F4E881F9810193F9839F
:10097000E88306C0E885F985802F0995892B31F435
:100980008E819F8101969F838E8302C00FEF1FEFA0
:10099000C801DF91CF911F910F910895FA01AA2705
:1009A000283051F1203181F1E8946F936E7F6E5FB2
:1009B0007F4F8F4F9F4FAF4FB1E03ED0B4E03CD060
:1009C000670F781F891F9A1FA11D680F791F8A1F43
:1009D000911DA11D6A0F711D811D911DA11D20D0AA
:1009E00009F468943F912AE0269F11243019305D64
:1009F0003193DEF6CF010895462F4770405D419355
:100A0000B3E00FD0C9F7F6CF462F4F70405D4A33A1
:100A100018F0495D31FD4052419302D0A9F7EACF69
:100A2000B4E0A6959795879577956795BA95C9F798
:100A300000976105710508959B01AC010A2E06948B
:100A40005795479537952795BA95C9F7620F731F44
:100A5000841F951FA01D08952F923F924F925F9281
:100A60006F927F928F929F92AF92BF92CF92DF92BE
:100A7000EF92FF920F931F93CF93DF93CDB7DEB723
:100A8000CA1BDB0B0FB6F894DEBF0FBECDBF0994B7
:100A90002A88398848885F846E847D848C849B840E
:100AA000AA84B984C884DF80EE80FD800C811B811C
:100AB000AA81B981CE0FD11D0FB6F894DEBF0FBE4B
:0A0AC000CDBFED010895F894FFCFBB
:100ACA002A72696E672A0A005374617274696E67C2
:100ADA002E2E2E0A0D0021287E50494E4420262013
:100AEA003078343029002E2E2F4173736572744783
:100AFA0043433634342E63002564200A0D0074699A
:100B0A006D653C31300000000003000000005E000B
:100B1A007A0000007461736B33007461736B320086
:100B2A00417373657274696F6E206661696C65647E
:100B3A003A20282573292C2066696C652025732C98
:100B4A00206C696E652025642E0A004173736572F4
:100B5A0074696F6E206661696C65643A2028257332
:100B6A00292C2066756E6374696F6E2025732C209C
:100B7A0066696C652025732C206C696E6520256476
:040B8A002E0A00002F
:00000001FF
